:100000000C9434000C9451000C9451000C94510049
:100010000C9451000C9451000C9451000C94130159
:100020000C9451000C9451000C9451000C94E2007B
:100030000C9451000C9451000C94B1000C9451009C
:100040000C9451000C9451000C9451000C945100EC
:100050000C9451000C9451000C9451000C945100DC
:100060000C9451000C94510011241FBECFEFD8E026
:10007000DEBFCDBF11E0A0E0B1E0EEEAF6E002C0E5
:1000800005900D92AC31B107D9F711E0ACE1B1E0C8
:1000900001C01D92A132B107E1F70E9468010C94E2
:1000A00055030C940000CF93DF93EC0190917C00FA
:1000B000957E956090937C0080917A008064809317
:1000C0007A0080917A0086FDFCCF60917800709173
:1000D000790080E090E00E94640220E030E040E897
:1000E00054E40E94F20220E030EC4FE754E40E9416
:1000F000FC016C837D838E839F838A8D9B8D8230F0
:10010000910561F08330910599F00197C9F416BC0F
:1001100080916E00826080936E0016C01092850000
:100120001092840080916F00826080936F000CC0F9
:100130001092B2008091700082608093700004C0C1
:1001400081E090E00E94550378949FB7F8948091E5
:100150001E019FBF8823C9F310921E01DF91CF912A
:1001600008951F920F920FB60F9211242F933F9371
:100170008F939F9380911C0190911D010196909304
:100180001D0180931C0180911E01813091F020910E
:100190001C0130911D0180911F01909120012817B1
:1001A000390738F081E080931E0110921D011092F2
:1001B0001C019F918F913F912F910F900FBE0F9037
:1001C0001F9018951F920F920FB60F9211242F9324
:1001D0003F938F939F9380911C0190911D010196F5
:1001E00090931D0180931C0180911E01813091F03C
:1001F00020911C0130911D0180911F0190912001DF
:100200002817390738F081E080931E0110921D01F4
:1002100010921C019F918F913F912F910F900FBED3
:100220000F901F9018951F920F920FB60F921124E6
:100230002F933F938F939F9380911C0190911D0169
:10024000019690931D0180931C0180911E018130C5
:1002500091F020911C0130911D0180911F0190911E
:1002600020012817390738F081E080931E01109291
:100270001D0110921C019F918F913F912F910F9022
:100280000FBE0F901F901895FC01ACE7B0E08C9169
:10029000806C8C93AAE7B0E08C9187688C93178A66
:1002A000168A85B5836085BD21E030E0318F208FCF
:1002B0008AE090E09093200180931F0184B58260D2
:1002C00084BD89EF87BD338F228F80E090E0089551
:1002D000CF92DF92EF92FF9280E091E00E94440182
:1002E000C12CD12C760160E070E0CB01609300015D
:1002F00070930101809302019093030180E091E0EB
:100300000E9453008FEFC81AD80AE80AF80AC701FA
:10031000B6010E9464022FE632E143E05BE30E94F3
:10032000F20220E030E0A9010E949801DFCF50588E
:10033000BB27AA270ED01CC10DD130F012D120F05E
:1003400031F49F3F11F41EF402C10EF4E095E7FB77
:10035000F8C0E92F1ED180F3BA176207730784072C
:10036000950718F071F49EF536C10EF4E0950B2E4A
:10037000BA2FA02D0B01B90190010C01CA01A001F7
:100380001124FF27591B99F0593F50F4503E68F152
:100390001A16F040A22F232F342F4427585FF3CF93
:1003A000469537952795A795F0405395C9F77EF464
:1003B0001F16BA0B620B730B840BBAF09150A1F0AD
:1003C000FF0FBB1F661F771F881FC2F70EC0BA0F33
:1003D000621F731F841F48F4879577956795B795BB
:1003E000F7959E3F08F0B3CF9395880F08F09927B3
:1003F000EE0F9795879508950CD0BAC0B2D040F013
:10040000A9D030F021F45F3F19F09BC05111E4C036
:100410009EC0BFD098F39923C9F35523B1F3951B20
:10042000550BBB27AA2762177307840738F09F5F15
:100430005F4F220F331F441FAA1FA9F333D00E2E84
:100440003AF0E0E830D091505040E695001CCAF7F1
:1004500029D0FE2F27D0660F771F881FBB1F2617B6
:1004600037074807AB07B0E809F0BB0B802DBF0189
:10047000FF2793585F4F2AF09E3F510568F061C0F7
:10048000ABC05F3FECF3983EDCF3869577956795BC
:10049000B795F7959F5FC9F7880F911D969587953A
:1004A00097F90895E1E0660F771F881FBB1F621759
:1004B00073078407BA0720F0621B730B840BBA0B17
:1004C000EE1F88F7E0950895E89409C097FB3EF485
:1004D00090958095709561957F4F8F4F9F4F992391
:1004E000A9F0F92F96E9BB279395F695879577950F
:1004F0006795B795F111F8CFFAF4BB0F11F460FFCF
:100500001BC06F5F7F4F8F4F9F4F16C0882311F026
:1005100096E911C0772321F09EE8872F762F05C03A
:10052000662371F096E8862F70E060E02AF09A95D5
:10053000660F771F881FDAF7880F9695879597F9CA
:10054000089597F99F6780E870E060E008959FEF55
:1005500080EC089500240A9416161706180609065A
:10056000089500240A941216130614060506089529
:10057000092E0394000C11F4882352F0BB0F40F4B1
:10058000BF2B11F460FF04C06F5F7F4F8F4F9F4FF1
:10059000089557FD9058440F551F59F05F3F71F073
:1005A0004795880F97FB991F61F09F3F79F08795DA
:1005B0000895121613061406551FF2CF4695F1DF63
:1005C00008C0161617061806991FF1CF86957105F3
:1005D000610508940895E894BB2766277727CB0127
:1005E00097F908950BD0C4CFB5DF28F0BADF18F023
:1005F000952309F0A6CFABCF1124EECFCADFA0F32D
:10060000959FD1F3950F50E0551F629FF001729FA7
:10061000BB27F00DB11D639FAA27F00DB11DAA1FC6
:10062000649F6627B00DA11D661F829F2227B00D13
:10063000A11D621F739FB00DA11D621F839FA00D9E
:10064000611D221F749F3327A00D611D231F849FEE
:10065000600D211D822F762F6A2F11249F57504045
:100660008AF0E1F088234AF0EE0FFF1FBB1F661FE0
:10067000771F881F91505040A9F79E3F510570F099
:1006800060CFAACF5F3FECF3983EDCF38695779579
:100690006795B795F795E7959F5FC1F7FE2B880F94
:0E06A000911D9695879597F90895F894FFCFD0
:1006AE000000000000000000000000000AD7233CFC
:0C06BE000200010000000000000000002D
:00000001FF
